:020000020000FC
:100000006BC16AC169C168C167C136C01BC02CC061
:1000100063C111C061C105C05FC15EC15DC15CC18A
:100020005BC10F930FB70F93BB2009F0BA940F91E8
:100030000FBF0F9118950F930FB70F930F910FBF2D
:100040000F9118950F930FB70F930091800009BD82
:100050000091810008BD00270EBD0DBD0CBDFF271E
:100060000F910FBF0F9118950F930FB70F93DD9856
:100070000F910FBF0F9118950F930FB70F931F9309
:1000800004B515B500937500109374001F910F917E
:100090000FBF0F9118957894109171000091720024
:1000A000011770F4101B10937F00002700937E004F
:1000B00000918200002391F001E00093870016C0B8
:1000C000011B00937F00002700937E0000918200B7
:1000D000002341F000E0009387000DC000E0009392
:1000E000870004C001E00093870005C00091710003
:1000F0000F3E30F00BC0009172000F3E20F006C0A2
:100100000F3960F012C00F3948F00FC0DC98009131
:100110008400013009F076D029D007C0DC9A009124
:100120008400013009F06ED021D022272093830073
:10013000089522273327369A349BFECF05B1369A8D
:10014000349BFECF15B1010F231F369A349BFECF8F
:1001500015B1010F231F369A349BFECF15B1010F45
:10016000231F26950795269507950895DB9804E3A8
:100170000A95F1F7DB9A089508E010E73117200798
:1001800010F4202F312F0FE010E03117200710F06E
:10019000202F312F089500917600109177003117AC
:1001A000200710F4202F312F08950091780010912E
:1001B00079003117200718F0202F312F3A95089534
:1001C00007E010ED3117200710F4202F312F08958C
:1001D00007E018E03117200710F4202F312F089581
:1001E0000FE010EA3117200718F0202F312F3A9531
:1001F000089500E118E63117200718F0202F312F5D
:100200003A9508950FEF22E12A95F1F700000000DA
:1002100000000000000000000A95A9F708950FEF04
:100220001FEF20E12A95F1F71A95D9F70A95C1F742
:1002300008950FEF11ED21E02A95F1F71A95D9F7FE
:100240000A95C1F7089506EF0000000000000000C5
:100250000000000000000000000000000A95A1F767
:100260000895CF99FECF7CD0F8941091750020911D
:10027000740078941093810020938000B299F1CF9C
:100280000895CDDFDA98CBDFDA9A0895002700933E
:1002900087000FEFB02ECDDFBB2059F0B299FBCF16
:1002A00010918700139510938700DA98B8DFDA9AD7
:1002B000F3CF0895E199FECF55275CBB4EBB8DBBB4
:1002C000E29AE19A0895E199FECF4EBBE09A5CB3C1
:1002D00050FDFDCF8DB3089501E00EBF0FE50DBFBA
:1002E000002700BF05E003BF01E009BF00E00FBD2C
:1002F00000E002BD06E20CB90BE00093800008EBC1
:10030000009381000091800009BD0091810008BD2B
:1003100001E10BBD00E30ABD00E807B906E806B934
:1003200000E103B901E001B9002708B9DE98D69AC7
:10033000DC98D49ADB9AD39ADD98D59AD198D09844
:10034000BA98C29AD99AD29ABB24FFEF0027009399
:100350007F0000937E0000938700009383000BC012
:100360007894CF9BFECFDD9A789402E80EBDFF23F0
:10037000F1F7FFEF0895B299C2C0DA98B29BFECFB1
:100380000FEFB02E7894BB2009F492C0CF9BFBCF27
:1003900049E081E08FDF43DFDA9A63DF0091740088
:1003A00010917500185B0B4060F046E0809174007E
:1003B00081DF47E0809175007DDF40E181E07ADFF9
:1003C0000BC043E08091740075DF44E080917500BC
:1003D00071DF40E180E06EDF54DF53DF42DF0091E8
:1003E000740010917500185B0B4048F046E0809156
:1003F000740060DF47E0809175005CDF08C043E077
:100400008091740057DF44E08091750053DF39DF3D
:1004100038DF37DF26DFF894009174001091750003
:10042000789443E050DF282F44E04DDF382F131B32
:10043000020B069517952091740030917500311BC1
:10044000200B10F427E038E0C3DE4BE0822F32DFD0
:100450004CE0832F2FDFF8942091740030917500C9
:10046000789446E030DF082F47E02DDF182F131B6C
:10047000020B06951795310F201F10F420E138E686
:10048000B8DE4EE0822F16DF4FE0832F13DFF9DE58
:10049000F8DEF7DEF6DEFADE1091870041E1812F0B
:1004A00009DFDA980EE3B02EBB20F1F7DA9A27C005
:1004B00049E080E0FFDEB3DEDA9AE8DE00918700F3
:1004C00000FD02C0002701C001E040E1802FF2DE04
:1004D000D8DED7DEDBDE0091870041E1802FEADE47
:1004E000D0DECFDECEDED2DE0091870042E1802F6B
:1004F000E1DEDA980EE3B02EBB20F1F7DA9A02E0E3
:1005000003BF789446E0DFDE8093780047E0DBDECF
:100510008093790043E0D7DE8093760044E0D3DE19
:10052000809377004BE0CFDE80937B004CE0CBDE06
:1005300080937A004EE0C7DE80937C004FE0C3DEFC
:1005400080937D0040E1BFDE8093820041E1BBDE0D
:100550008093850042E1B7DE8093860049E0B3DEF8
:1005600080938400813009F087C00FE000938800F9
:10057000F7DE209174003091750000917B0010919E
:100580007A003117200708F420C000917C001091F8
:100590007D0031172007C8F400918700002359F42B
:1005A00000917E0010917F00311B200B10F427E09A
:1005B00038E0F1DD0AC000917E0010917F00310F1C
:1005C000201F10F420E138E6F0DD20938000309306
:1005D0008100DE9817DE16DE15DE14DEAADD00933C
:1005E00071000027C99901E000938B00DE9A0ADEB2
:1005F00009DE08DE07DE9DDD009372000027C99941
:1006000001E000938A0047DD00918B00002359F040
:1006100000918A00002339F0002700937F000093A7
:100620007E00DA9AA2CF20917E0030917F00DA9886
:1006300000918500002359F0013081F0033099F0DA
:10064000330F221F20937E0030937F008ECF26959C
:10065000379520937E0030937F0087CF20937E00D4
:1006600030937F0082CF330F221F330F221F20933E
:100670007E0030937F0079CF76DE0EE5B02EDE98D7
:10068000C1DDC0DDBFDDBEDDBDDD53DD009371002A
:100690000027C99901E000938B00DE9AB3DDB2DD3B
:1006A000B1DDB0DDAFDD45DD009372000027C999F3
:1006B00001E000938A00EFDC00918B00002359F0E9
:1006C00000918A00002339F0002700937F000093F7
:1006D0007E00DA9A56C00027DA9820917E00309189
:1006E0007F0000918500002331F4889420937E00E0
:1006F00030937F0021C0023051F4330F221F8894C1
:10070000330F221F20937E0030937F0015C00330EB
:1007100069F4330F221F8894330F221F8894330FFC
:10072000221F20937E0030937F0006C0330F221FCC
:1007300020937E0030937F0000918700002369F0B2
:1007400020917E0030917F000BE018EB310F201FCD
:1007500010F42FE030EA44DD0CC000917E001091CF
:100760007F002BE038EB311B200B10F427E030ED3D
:1007700027DD36DD2093800030938100BB20F1F728
:100780007BCF00918600002309F4F8CF033039F4C1
:100790002BE02093800038EB30938100EFCF0130C5
:1007A00041F520918000309181000BE01CEB311766
:1007B000200750F014E00027311B200B01DD2093AF
:1007C000800030938100DACF0BE014EB3117200763
:1007D00038F00BE018EB2093800030938100CECFEF
:1007E00014E00027310F201F2093800030938100F8
:1007F000C5CF20918000309181000BE010EC3117C3
:10080000200748F018E00027311B200B20938000C0
:1008100030938100B3CF0BE010EB3117200738F095
:100820000BE018EB2093800030938100A7CF18E0F5
:100830000027310F201F20938000309381009ECF2E
:00000001FF
